:020000040000FA
:04080000F2EF07F01C
:1008100003B213EF05F0F2B431EF05F09EB039EFFB
:1008200005F09EB241EF05F0F2A81AEF04F0F2B223
:1008300025EF04F0F2A620EF04F0F2B022EF04F06E
:10084000A1EF07F0F296F290FF00CD90F2929EA0F9
:100850002FEF04F00101533F2FEF04F0542BAEC1F2
:10086000B2F1AFC1B3F1B0C1B4F1B1C1B5F1AAC138
:10087000AEF1ABC1AFF1ACC1B0F1ADC1B1F1A6C148
:10088000AAF1A7C1ABF1A8C1ACF1A9C1ADF1A2C158
:10089000A6F1A3C1A7F1A4C1A8F1A5C1A9F19EC168
:1008A000A2F19FC1A3F1A0C1A4F1A1C1A5F19AC178
:1008B0009EF19BC19FF19CC1A0F19DC1A1F196C188
:1008C0009AF197C19BF198C19CF199C19DF1CECF4E
:1008D00096F1CFCF97F153C198F154C199F1CF6AF6
:1008E000CE6A0101536B546B9E90CD800FBC0F8E6E
:1008F0000FBA7EEF04F00F8AA1EF07F00F8C0FBE46
:10090000BAEF04F096C19AF197C19BF198C19CF19E
:1009100099C19DF19AC19EF19BC19FF19CC1A0F12B
:100920009DC1A1F19EC1A2F19FC1A3F1A0C1A4F1FB
:10093000A1C1A5F1A2C1A6F1A3C1A7F1A4C1A8F1CB
:10094000A5C1A9F1A6C1AAF1A7C1ABF1A8C1ACF19B
:10095000A9C1ADF1AAC1AEF1ABC1AFF1ACC1B0F16B
:10096000ADC1B1F1AEC1B2F1AFC1B3F1B0C1B4F13B
:10097000B1C1B5F101015E6B5F6B606B616B96514C
:100980005E2797515F2398516023995161239A51B3
:100990005E279B515F239C5160239D5161239E5193
:1009A0005E279F515F23A0516023A1516123A25173
:1009B0005E27A3515F23A4516023A5516123A65153
:1009C0005E27A7515F23A8516023A9516123AA5133
:1009D0005E27AB515F23AC516023AD516123AE5113
:1009E0005E27AF515F23B0516023B1516123B251F3
:1009F0005E27B3515F23B4516023B5516123D89072
:100A00000101613360335F335E33D890010161339C
:100A100060335F335E33D8900101613360335F33FD
:100A20005E33A1EF07F00392ABB2AB98AB88030142
:100A300003EE00F080517F0BE92604C0EFFF802B0E
:100A40008151805D700BD8A48B8200008051815D44
:100A5000700BD8A48B9281518019D8B40790A1EF64
:100A600007F0F2940101453FA1EF07F0462BA1EFFB
:100A700007F09E900101533FA1EF07F0542BA1EF27
:100A800007F09E92040062A146EF05F0077C07ACD8
:100A900061EF05F0C274C2B45BEF05F0C3CFB3F5EC
:100AA000C4CFB4F50501D890B433B333D890B43380
:100AB000B33362EF05F0C3CF55F1C4CF56F162EF07
:100AC00005F0C28207B4CFEF05F047C14BF148C132
:100AD0004CF149C14DF14AC14EF15EC162F15FC1B5
:100AE00063F160C164F161C165F196C1B6F197C16E
:100AF000B7F198C1B8F199C1B9F19AC1BAF19BC1E6
:100B0000BBF19CC1BCF19DC1BDF19EC1BEF19FC1B5
:100B1000BFF1A0C1C0F1A1C1C1F1A2C1C2F1A3C185
:100B2000C3F1A4C1C4F1A5C1C5F1A6C1C6F1A7C155
:100B3000C7F1A8C1C8F1A9C1C9F1AAC1CAF1ABC125
:100B4000CBF1ACC1CCF1ADC1CDF1AEC1CEF1AFC1F5
:100B5000CFF1B0C1D0F1B1C1D1F1B2C1D2F1B3C1C5
:100B6000D3F1B4C1D4F1B5C1D5F1B3C5B5F5B4C5B0
:100B7000B6F5B5C5B7F5B6C5B8F5010155515B2752
:100B800056515C23E86A5D230E2ECFEF05F05CC161
:100B900057F15DC158F15B6B5C6B5D6B078E0201B9
:100BA000002FA1EF07F03C0E006F00C10CF101C156
:100BB0000DF102C10EF103C10FF104C110F105C125
:100BC00011F106C112F107C113F108C114F109C1F5
:100BD00015F10AC116F10BC117F134C135F1050148
:100BE0002F51000AD8B4A0EF06F005012F51010AD9
:100BF000D8B42AEF06F005012F51020AD8B46BEFE2
:100C000006F005012F51030AD8B46BEF06F0050179
:100C10002F51040AD8B46BEF06F005012F51050AD5
:100C2000D8B46BEF06F005012F51060AD8B46BEF6C
:100C300006F005012F51070AD8B46BEF06F0050145
:100C40002F51320AD8B428EF06F02F6BA0EF06F030
:100C5000A0EF06F00501536735EF06F0546735EF56
:100C600006F0556735EF06F0566739EF06F0A0EF4E
:100C700006F057C500F158C501F159C502F15AC532
:100C800003F10101010E046F000E056F000E066FE7
:100C9000000E076F2DEC20F000C157F501C158F58B
:100CA00002C159F503C15AF500675EEF06F001670E
:100CB0005EEF06F002675EEF06F00367A0EF06F056
:100CC00053C557F554C558F555C559F556C55AF588
:100CD0000F88A0EF06F00501306771EF06F0A0EF76
:100CE00006F00FBE86EF06F010A08BEF06F00101B4
:100CF000476782EF06F0486782EF06F0496782EFA8
:100D000006F04A6786EF06F08BEF06F007AE8BEF32
:100D100006F09DEF06F00501312FA0EF06F03C0E26
:100D2000316F302FA0EF06F00101000E626FE00E70
:100D3000636FA50E646F010E656F0501306B0F8840
:100D40000501626B33B7A6EF06F062810CC100F1BA
:100D50000DC101F10EC102F10FC103F110C104F187
:100D600011C105F112C106F113C107F114C108F157
:100D700015C109F116C10AF117C10BF135C134F1E2
:100D800000C10CF101C10DF102C10EF103C10FF15F
:100D900004C110F105C111F106C112F107C113F12F
:100DA00008C114F109C115F10AC116F10BC117F1FF
:100DB00034C135F101018A67E5EF06F08B67E5EF95
:100DC00006F08C67E5EF06F08D67E9EF06F019EFA6
:100DD00007F08EC100F18FC101F190C102F191C104
:100DE00003F10101010E046F000E056F000E066F86
:100DF000000E076F2DEC20F000C18EF101C18FF1C4
:100E000002C190F103C191F100670EEF07F0016795
:100E10000EEF07F002670EEF07F0036719EF07F018
:100E20008AC18EF18BC18FF18CC190F18DC191F18E
:100E30000F80D57ED5BE69D0D6CF47F1D7CF48F148
:100E400045C149F1E86AE8CF4AF1109047C100F185
:100E500048C101F149C102F14AC103F101010A0E81
:100E6000046F000E056F000E066F000E076F2DEC6D
:100E700020F003AF1080010154A74BEF07F00F9A49
:100E80000F9C0F9E0101000E5E6F600E5F6F3D0EA6
:100E9000606F080E616F010147BF5BEF07F04867A5
:100EA0005BEF07F049675BEF07F04A675BEF07F01E
:100EB000F28880EF07F0F2985E6B5F6B606B616B9E
:100EC000966B976B986B996B9A6B9B6B9C6B9D6BFE
:100ED0009E6B9F6BA06BA16BA26BA36BA46BA56BAE
:100EE000A66BA76BA86BA96BAA6BAB6BAC6BAD6B5E
:100EF000AE6BAF6BB06BB16BB26BB36BB46BB56B0E
:100F0000D76AD66A0101456B466B0CC100F10DC171
:100F100001F10EC102F10FC103F110C104F111C1C1
:100F200005F112C106F113C107F114C108F115C191
:100F300009F116C10AF117C10BF135C134F1A1EF66
:100F400007F002C0E0FF005001C0D8FF1000A6B2B9
:100F5000A7EF07F00CC0A9FF0BC0A8FFA69EA69C98
:100F6000A684F29E550EA76EAA0EA76EA682F28EDA
:100F7000A694A6B2B9EF07F00C2A1200A96EA69E9D
:100F8000A69CA680A8500C2A120004012C0E826F89
:100F9000CBEC0AF028EC21F00C50BEEC07F0E8CFC7
:100FA00000F10C50BEEC07F0E8CF01F101AFDEEF2D
:100FB00007F00101FF0E026FFF0E036FCBEC20F074
:100FC0002967EAEF07F00401200E826FCBEC0AF0EC
:100FD000EFEF07F004012D0E826FCBEC0AF0F5EC79
:100FE0001EF01200076A0F6A106A0F010D0EC16E23
:100FF000860EC06E030EC26E0F01680E896E130E50
:10100000926E080E8A6EF30E936E8B6A900E946E3B
:10101000C80EBEEC07F0E8CFE8FF1098E8A01088F3
:1010200010A805D00E0E156E8E0E166E04D00F0E83
:10103000156E8F0E166EA7EC21F0F18EF19E0E6AE2
:1010400001015B6B5C6B5D6B576B586BF29A010136
:10105000476B486B496B4A6B4B6B4C6B4D6B4E6BE4
:101060004F6B506B516B526B456B466BD76AD66AB0
:101070000F01280ED56EF28A9D90B00ECD6E010143
:101080005E6B5F6B606B616B626B636B646B656BFC
:10109000666B676B686B696B536B546BCF6ACE6A18
:1010A0000F9A0F9C0F9E9D80760ECA6E9D82020144
:1010B0003C0E006FCC6A160EBEEC07F0E8CF00F1D4
:1010C000170EBEEC07F0E8CF01F1180EBEEC07F0EA
:1010D000E8CF02F1190EBEEC07F0E8CF03F10101F1
:1010E00003AF8DEF08F028EC21F0160E0C6E00C156
:1010F0000BF0A7EC07F0170E0C6E01C10BF0A7EC7C
:1011000007F0180E0C6E02C10BF0A7EC07F0190ED9
:101110000C6E03C10BF0A7EC07F000C18AF101C10E
:101120008BF102C18CF103C18DF100C18EF101C1BF
:101130008FF102C190F103C191F11A0EBEEC07F0DC
:10114000E8CF00F11B0EBEEC07F0E8CF01F11C0E5A
:10115000BEEC07F0E8CF02F11D0EBEEC07F0E8CFC1
:1011600003F1010103AFE3EF08F028EC21F01A0EC0
:101170000C6E00C10BF0A7EC07F01B0E0C6E01C14A
:101180000BF0A7EC07F01C0E0C6E02C10BF0A7ECE5
:1011900007F01D0E0C6E03C10BF0A7EC07F01A0E42
:1011A000BEEC07F0E8CF00F11B0EBEEC07F0E8CF75
:1011B00001F11C0EBEEC07F0E8CF02F11D0EBEECF3
:1011C00007F0E8CF03F100C192F101C193F102C130
:1011D00094F103C195F1240EAC6E900EAB6E240E0B
:1011E000AC6E080EB86E000EB06E1F0EAF6E04012E
:1011F000806B816B0F01900EAB6E0F019D8A030116
:10120000806B816BC26B8B922FEC26F02FEC26F05B
:101210008BEC27F00EEC24F0200EBEEC07F0E8CFAC
:101220002FF505012F51FF0AD8A41EEF09F02F6BEF
:10123000200E0C6E2FC50BF0A7EC07F00501010E78
:10124000306F3C0E316F250EBEEC07F0E8CF00F199
:10125000260EBEEC07F0E8CF01F1270EBEEC07F03A
:10126000E8CF02F1280EBEEC07F0E8CF03F1010150
:1012700003AF55EF09F028EC21F0250E0C6E00C1EC
:101280000BF0A7EC07F0260E0C6E01C10BF0A7ECDB
:1012900007F0270E0C6E02C10BF0A7EC07F0280E2A
:1012A0000C6E03C10BF0A7EC07F000C153F501C1B0
:1012B00054F502C155F503C156F500C157F501C1FA
:1012C00058F502C159F503C15AF5290EBEEC07F0D5
:1012D000E8CF5BF505015C515B5DD8A05BC55CF5B3
:1012E00005012F51020A0EE181B882EF09F00501D4
:1012F0005C2F7FEF09F05BC55CF582EF09F081BAE6
:10130000CAEF27F0210EBEEC07F0E8CF00F1220E65
:10131000BEEC07F0E8CF01F1230EBEEC07F0E8CFFA
:1013200002F1240EBEEC07F0E8CF03F1010103AF98
:10133000C8EF09F028EC21F0210E0C6E00C10BF073
:10134000A7EC07F0220E0C6E01C10BF0A7EC07F022
:10135000230E0C6E02C10BF0A7EC07F0240E0C6EEE
:1013600003C10BF0A7EC07F0210EBEEC07F0E8CFAD
:1013700000F1220EBEEC07F0E8CF01F1230EBEEC27
:1013800007F0E8CF02F1240EBEEC07F0E8CF03F13E
:1013900000C15DF501C15EF502C15FF503C160F5F5
:1013A00056EC23F058EC22F0B0EC21F005012F515F
:1013B000030A12E005012F51040A1DE005012F5117
:1013C000050A24E005012F51060A32E005012F51DC
:1013D000070A38E02BEF0AF0ACC500F101010F0E4F
:1013E000001701010051000A36E001010051050A11
:1013F00032E028EF0AF0ACC500F101010F0E001732
:1014000001010051000A27E028EF0AF00501AC5164
:10141000000A21E00501AC51150A1DE00501AC519F
:10142000300A19E00501AC51450A15E028EF0AF031
:101430000501AC51000A0FE00501AC51300A0BE088
:1014400028EF0AF00501AC51000A05E028EF0AF088
:1014500081BACAEF27F007900001F28EF28C07B034
:1014600076EF1DF00FB055EF18F00FB819EF12F02E
:101470000301805181197F0BD8B476EF1DF013EE74
:1014800000F081517F0BE126812BE7CFE8FFE00BD5
:10149000D8B476EF1DF023EE82F0C2513F0BD9266F
:1014A000E7CFDFFFC22BDF50780AD8A476EF1DF01C
:1014B00007808EC100F18FC101F190C102F191C18D
:1014C00003F10101040E046F000E056F000E066F9C
:1014D000000E076F2DEC20F000AF78EF0AF001014D
:1014E000030E8E6F000E8F6F000E906F000E916FC7
:1014F00003018251720AD8B455EF18F08251520A92
:10150000D8B455EF18F08251750AD8B455EF18F0D9
:101510008251630AD8B430EF1AF08251690AD8B404
:1015200010EF15F082517A0AD8B423EF16F08251E9
:10153000490AD8B4AFEF14F08251500AD8B4CDEFB5
:1015400013F08251700AD8B410EF14F08251540A8B
:10155000D8B43BEF14F08251740AD8B481EF14F080
:1015600082516D0AD8B4DFEF0AF082514D0AD8B427
:10157000F8EF0AF08251730AD8B485EF17F0825160
:10158000530AD8B4EAEF17F082514C0AD8B487EF67
:101590000BF067EF1AF0040114EE00F080517F0B9E
:1015A000E12682C4E7FF802B120004010D0E826F3A
:1015B000CBEC0AF00A0E826FCBEC0AF012000401A9
:1015C0006D0E826FCBEC0AF003018351300AD8B460
:1015D00037EF0BF003018351310AD8B44AEF0BF017
:1015E00003018351320AD8B45DEF0BF067EF1AF0B4
:1015F00004014D0E826FCBEC0AF069EC21F084C33C
:1016000031F185C332F186C333F10101296B76ECE8
:1016100021F0EDEC20F003018351300AD8B41FEF24
:101620000BF003018351310AD8B427EF0BF003010B
:101630008351320AD8B42FEF0BF067EF1AF0FD0E8A
:101640000C6E00C10BF0A7EC07F037EF0BF0FE0EAD
:101650000C6E00C10BF0A7EC07F04AEF0BF0FF0E89
:101660000C6E00C10BF0A7EC07F05DEF0BF004016E
:10167000300E826FCBEC0AF004012C0E826FCBECA3
:101680000AF028EC21F0FD0EBEEC07F0E8CF00F1E7
:101690006EEF0BF00401310E826FCBEC0AF0040107
:1016A0002C0E826FCBEC0AF028EC21F0FE0EBEEC83
:1016B00007F0E8CF00F16EEF0BF00401320E826FFD
:1016C000CBEC0AF028EC21F004012C0E826FCBEC5D
:1016D0000AF0FF0EBEEC07F0E8CF00F1CBEC20F0F3
:1016E00031C182F40401300E8227CBEC0AF032C102
:1016F00082F40401300E8227CBEC0AF033C182F46D
:101700000401300E8227CBEC0AF065EF1AF00301DA
:101710008351300AD8B4F2EF0EF003018351310A3D
:10172000D8B41FEF10F003018351320AD8B48DEF03
:1017300010F003018351330AD8B49DEF10F0030178
:101740008351340AD8B4ADEF10F003018351350A48
:10175000D8B41EEF12F003018351360AD8B44CEF0F
:1017600012F003018351370AD8B454EF0EF003018D
:101770008351460AD8B472EF11F0030183514D0A28
:10178000D8B4CDEF0CF0030183516D0AD8B4E7EF64
:101790000CF0030183515A0AD8B499EF0FF00301FA
:1017A0008351490AD8B44CEF13F003018351500A16
:1017B000D8B47EEF12F003018351540AD8B4F7EF86
:1017C00012F003018351630AD8B407EF0DF003014F
:1017D0008351430AD8B4FFEF0DF003018351730A1C
:1017E000D8B405EF0DF003018351610AD8B41AEFA4
:1017F0000CF003018351650AD8B442EF0FF00301E6
:101800008351450AD8B450EF0FF003018351620AA7
:10181000D8B45EEF0FF003018351420AD8B46CEFE5
:101820000FF003018351760AD8B47AEF0FF0D8A4F1
:1018300067EF1AF004014C0E826FCBEC0AF0040142
:10184000610E826FCBEC0AF058EC22F004012C0EF2
:10185000826FCBEC0AF028EC21F0ABC500F101015E
:10186000CBEC20F031C182F40401300E8227CBECA6
:101870000AF032C182F40401300E8227CBEC0AF068
:1018800033C182F40401300E8227CBEC0AF004014C
:101890002C0E826FCBEC0AF028EC21F0ACC500F1E5
:1018A0000101CBEC20F031C182F40401300E82271B
:1018B000CBEC0AF032C182F40401300E8227CBEC6B
:1018C0000AF033C182F40401300E8227CBEC0AF017
:1018D00004012C0E826FCBEC0AF028EC21F0ADC590
:1018E00000F10101CBEC20F031C182F40401300E93
:1018F0008227CBEC0AF032C182F40401300E822739
:10190000CBEC0AF033C182F40401300E8227CBEC19
:101910000AF004012C0E826FCBEC0AF028EC21F0C7
:10192000AEC500F10101CBEC20F031C182F404011D
:10193000300E8227CBEC0AF032C182F40401300E63
:101940008227CBEC0AF033C182F40401300E8227E7
:10195000CBEC0AF004012C0E826FCBEC0AF028ECE1
:1019600021F0B2C500F10101CBEC20F031C182F4CD
:101970000401300E8227CBEC0AF032C182F404015C
:10198000300E8227CBEC0AF033C182F40401300E12
:101990008227CBEC0AF07AEF12F069EC21F084C3D5
:1019A00033F176EC21F0EDEC20F0200E0C6E00C14E
:1019B0000BF0A7EC07F000C12FF505012F51000A2D
:1019C00006E005012F51010A02E0F2EC22F00401C9
:1019D0004C0E826FCBEC0AF004014D0E826FCBEC03
:1019E0000AF004012C0E826FCBEC0AF028EC21F0F7
:1019F0002FC500F1CBEC20F033C182F40401300E8E
:101A00008227CBEC0AF07AEF12F0CAEF27F004013C
:101A10004C0E826FCBEC0AF00401630E826FCBECAC
:101A20000AF0B0EC21F004012C0E826FCBEC0AF02E
:101A30001CEC0DF07AEF12F028EC21F0B1C500F1AA
:101A40000101003B0F0E0017CBEC20F033C182F4F4
:101A50000401300E8227CBEC0AF0B1C500F1010180
:101A60000F0E01010017CBEC20F033C182F404010A
:101A7000300E8227CBEC0AF004012D0E826FCBECE6
:101A80000AF0B0C500F10101003B0F0E0017CBECCE
:101A900020F033C182F40401300E8227CBEC0AF02F
:101AA000B0C500F101010F0E01010017CBEC20F0D1
:101AB00033C182F40401300E8227CBEC0AF004011A
:101AC0002D0E826FCBEC0AF0AFC500F10101003B97
:101AD0000F0E0017CBEC20F033C182F40401300E5E
:101AE0008227CBEC0AF0AFC500F101010F0E010116
:101AF0000017CBEC20F033C182F40401300E8227B2
:101B0000CBEC0AF00401200E826FCBEC0AF0AEC5DC
:101B100000F10F0E01010017CBEC20F033C182F46D
:101B20000401300E8227CBEC0AF00401200E826FF4
:101B3000CBEC0AF0ADC500F101010101003B0F0E35
:101B40000017CBEC20F033C182F40401300E822761
:101B5000CBEC0AF0ADC500F101010F0E0101001739
:101B6000CBEC20F033C182F40401300E8227CBECA1
:101B70000AF004013A0E826FCBEC0AF0ACC500F11A
:101B80000101003B0F0E0017CBEC20F033C182F4B3
:101B90000401300E8227CBEC0AF0ACC500F1010144
:101BA0000F0E01010017CBEC20F033C182F40401C9
:101BB000300E8227CBEC0AF004013A0E826FCBEC98
:101BC0000AF0ABC500F10101003B0F0E0017CBEC92
:101BD00020F033C182F40401300E8227CBEC0AF0EE
:101BE000ABC500F101010F0E0017CBEC20F033C1A3
:101BF00082F40401300E8227CBEC0AF0120084C379
:101C0000E8FF0F0BE83AE8CFB1F585C3E8FF0F0B0B
:101C10000501B11387C3E8FF0F0BE83AE8CFB0F531
:101C200088C3E8FF0F0B0501B0138AC3E8FF0F0B51
:101C3000E83AE8CFAFF58BC3E8FF0F0B0501AF1310
:101C40008DC3E8FF0F0BE8CFAEF58FC3E8FF0F0B96
:101C5000E83AE8CFADF590C3E8FF0F0B0501AD13EF
:101C600092C3E8FF0F0BE83AE8CFACF593C3E8FF67
:101C70000F0B0501AC1395C3E8FF0F0BE83AE8CF53
:101C8000ABF596C3E8FF0F0B0501AB130BEC22F08D
:101C900004014C0E826FCBEC0AF00401430E826FFC
:101CA000CBEC0AF011EF0DF0078404014C0E826FAB
:101CB000CBEC0AF00401370E826FCBEC0AF0040182
:101CC0002C0E826FCBEC0AF005012E51130A06E0B0
:101CD00005012E51170A0DE0EFEF0EF00101000E85
:101CE000006F000E016F100E026F000E036F82EF87
:101CF0000EF00101000E006F000E016F000E026F6A
:101D0000010E036FCBEC20F02AC182F40401300EE7
:101D10008227CBEC0AF02BC182F40401300E82271B
:101D2000CBEC0AF02CC182F40401300E8227CBECFC
:101D30000AF02DC182F40401300E8227CBEC0AF0A8
:101D40002EC182F40401300E8227CBEC0AF02FC1A1
:101D500082F40401300E8227CBEC0AF030C182F409
:101D60000401300E8227CBEC0AF031C182F4040169
:101D7000300E8227CBEC0AF032C182F40401300E1F
:101D80008227CBEC0AF033C182F40401300E8227A3
:101D9000CBEC0AF004012C0E826FCBEC0AF00101AF
:101DA000100E006F000E016F000E026F000E036F29
:101DB000CBEC20F031C182F40401300E8227CBEC51
:101DC0000AF032C182F40401300E8227CBEC0AF013
:101DD00033C182F40401300E8227CBEC0AF0079461
:101DE0007AEF12F007848BEC27F028EC21F02DC558
:101DF00000F1CBEC20F004014C0E826FCBEC0AF02A
:101E00000401300E826FCBEC0AF004012C0E826FBD
:101E1000CBEC0AF031C182F40401300E8227CBEC06
:101E20000AF032C182F40401300E8227CBEC0AF0B2
:101E300033C182F40401300E8227CBEC0AF0040196
:101E40002C0E826FCBEC0AF028EC21F02EC500F1AD
:101E5000CBEC20F031C182F40401300E8227CBECB0
:101E60000AF032C182F40401300E8227CBEC0AF072
:101E700033C182F40401300E8227CBEC0AF00794C0
:101E80007AEF12F004014C0E826FCBEC0AF00401E1
:101E9000650E826FCBEC0AF0B2EC23F07AEF12F011
:101EA00004014C0E826FCBEC0AF00401450E826FE8
:101EB000CBEC0AF0C9EC23F07AEF12F004014C0EDF
:101EC000826FCBEC0AF00401620E826FCBEC0AF059
:101ED000F7EC23F07AEF12F004014C0E826FCBEC9A
:101EE0000AF00401420E826FCBEC0AF0E0EC23F022
:101EF0007AEF12F004014C0E826FCBEC0AF0040171
:101F0000760E826FCBEC0AF004012C0E826FCBECC4
:101F10000AF010A807D00401310E826FCBEC0AF052
:101F20007AEF12F00401300E826FCBEC0AF07AEFF8
:101F300012F004014C0E826FCBEC0AF004015A0E31
:101F4000826FCBEC0AF004012C0E826FCBEC0AF00E
:101F50008BEC27F028EC21F005012E51130A06E046
:101F600005012E51170A0DE0CAEF0FF00101000E16
:101F7000006F000E016F100E026F000E036FCAEFAC
:101F80000FF00101000E006F000E016F000E026FD6
:101F9000010E036F0101100E046F000E056F000E9D
:101FA000066F000E076F5EEC20F0CBEC20F02AC12C
:101FB00082F40401300E8227CBEC0AF02BC182F4AC
:101FC0000401300E8227CBEC0AF02CC182F404010C
:101FD000300E8227CBEC0AF02DC182F40401300EC2
:101FE0008227CBEC0AF02EC182F40401300E822746
:101FF000CBEC0AF02FC182F40401300E8227CBEC27
:102000000AF030C182F40401300E8227CBEC0AF0D2
:1020100031C182F40401300E8227CBEC0AF032C1C8
:1020200082F40401300E8227CBEC0AF033C182F433
:102030000401300E8227CBEC0AF07AEF12F007840D
:1020400004014C0E826FCBEC0AF00401310E826F5A
:10205000CBEC0AF004012C0E826FCBEC0AF025C504
:1020600000F126C501F127C502F128C503F10101E0
:10207000100E046F000E056F000E066F000E076F46
:102080005EEC20F0CBEC20F02AC182F40401300E8B
:102090008227CBEC0AF02BC182F40401300E822798
:1020A000CBEC0AF02CC182F40401300E8227CBEC79
:1020B0000AF02DC182F40401300E8227CBEC0AF025
:1020C0002EC182F40401300E8227CBEC0AF02FC11E
:1020D00082F40401300E8227CBEC0AF030C182F486
:1020E0000401300E8227CBEC0AF031C182F40401E6
:1020F000300E8227CBEC0AF032C182F40401300E9C
:102100008227CBEC0AF033C182F40401300E82271F
:10211000CBEC0AF007947AEF12F0078404014C0E1E
:10212000826FCBEC0AF00401320E826FCBEC0AF026
:10213000E5EC25F007947AEF12F0078404014C0EC9
:10214000826FCBEC0AF00401330E826FCBEC0AF005
:1021500042EC26F007942AEF10F0078404014C0E9D
:10216000826FCBEC0AF00401340E826FCBEC0AF0E4
:1021700004012C0E826FCBEC0AF069EC21F084C3D1
:102180002AF185C32BF186C32CF187C32DF188C3B7
:102190002EF189C32FF18AC330F18BC331F18CC387
:1021A00032F18DC333F10101296B76EC21F0EDECB6
:1021B00020F0100E046F000E056F000E066F000E6B
:1021C000076F3EEC20F000C121F501C122F502C1EC
:1021D00023F503C124F53EEC27F034C5ABF535C536
:1021E000ACF536C5ADF537C5AEF538C5AFF539C573
:1021F000B0F53AC5B1F51CEC0DF004012C0E826F60
:10220000CBEC0AF03BC500F13CC501F13DC502F144
:102210003EC503F10101000E046F000E056F010EB3
:10222000066F000E076F5EEC20F0CBEC20F0296704
:102230001CEF11F021EF11F004012D0E826FCBEC99
:102240000AF030C182F40401300E8227CBEC0AF090
:1022500031C182F40401300E8227CBEC0AF0040174
:102260002E0E826FCBEC0AF032C182F40401300EE4
:102270008227CBEC0AF033C182F40401300E8227AE
:10228000CBEC0AF004012C0E826FCBEC0AF028ECA8
:1022900021F03FC500F140C501F191EC1BF00401B4
:1022A0002C0E826FCBEC0AF028EC21F041C500F136
:1022B000CBEC20F031C182F40401300E8227CBEC4C
:1022C0000AF032C182F40401300E8227CBEC0AF00E
:1022D00033C182F40401300E8227CBEC0AF007945C
:1022E0007AEF12F069EC21F085C32AF186C32BF155
:1022F00087C32CF188C32DF189C32EF18AC32FF136
:102300008BC330F18CC331F18DC332F18EC333F105
:102310000101296B76EC21F0EDEC20F00101010EBA
:10232000046F000E056F000E066F000E076F2DEC98
:1023300020F0100E046F000E056F000E066F000EE9
:10234000076F3EEC20F000C129F501C12AF502C15A
:102350002BF503C12CF56CEC25F004014C0E826FBB
:10236000CBEC0AF00401460E826FCBEC0AF00401BC
:102370002C0E826FCBEC0AF025C500F126C501F1C9
:1023800027C502F128C503F10101100E046F000EEC
:10239000056F000E066F000E076F5EEC20F0CBECB1
:1023A00020F02AC182F40401300E8227CBEC0AF01F
:1023B0002BC182F40401300E8227CBEC0AF02CC131
:1023C00082F40401300E8227CBEC0AF02DC182F496
:1023D0000401300E8227CBEC0AF02EC182F40401F6
:1023E000300E8227CBEC0AF02FC182F40401300EAC
:1023F0008227CBEC0AF030C182F40401300E822730
:10240000CBEC0AF031C182F40401300E8227CBEC10
:102410000AF032C182F40401300E8227CBEC0AF0BC
:1024200033C182F40401300E8227CBEC0AF07AEF3C
:1024300012F00F9842EC26F067EF1AF004014C0EF0
:10244000826FCBEC0AF00401350E826FCBEC0AF000
:1024500004012C0E826FCBEC0AF028EC21F00784EB
:10246000B5C500F10794CBEC20F031C182F4040132
:10247000300E8227CBEC0AF032C182F40401300E18
:102480008227CBEC0AF033C182F40401300E82279C
:10249000CBEC0AF07AEF12F005EC26F028EC21F0F4
:1024A00033C500F1CBEC20F004014C0E826FCBEC75
:1024B0000AF00401360E826FCBEC0AF004012C0EF8
:1024C000826FCBEC0AF031C182F40401300E822716
:1024D000CBEC0AF032C182F40401300E8227CBEC3F
:1024E0000AF033C182F40401300E8227CBEC0AF0EB
:1024F0007AEF12F0D5EC0AF067EF1AF004014C0EF7
:10250000826FCBEC0AF00401500E826FCBEC0AF024
:1025100004012C0E826FCBEC0AF085C32AF186C32E
:102520002BF187C32CF188C32DF189C32EF18AC307
:102530002FF18BC330F18CC331F18DC332F18EC3D7
:1025400033F1010176EC21F0EDEC20F00301845130
:10255000530A0DE0030184514D0A38E00401780E5E
:10256000826FCBEC0AF0D5EC0AF067EF1AF00401A9
:10257000530E826FCBEC0AF0250E0C6E00C10BF0EF
:10258000A7EC07F0260E0C6E01C10BF0A7EC07F0CC
:10259000270E0C6E02C10BF0A7EC07F0280E0C6E94
:1025A00003C10BF0A7EC07F000C153F501C154F5CE
:1025B00002C155F503C156F500C157F501C158F5E3
:1025C00002C159F503C15AF55BEF13F004014D0E3A
:1025D000826FCBEC0AF0290E0C6E00C10BF0A7EC59
:1025E00007F000C15BF500C15CF55BEF13F004017F
:1025F0004C0E826FCBEC0AF00401540E826FCBECD0
:102600000AF004012C0E826FCBEC0AF084C32AF18D
:1026100085C32BF186C32CF187C32DF188C32EF11E
:1026200089C32FF18AC330F18BC331F18DC332F1ED
:102630008EC333F1010176EC21F0EDEC20F00101C5
:10264000000E046F000E056F010E066F000E076F7F
:102650003EEC20F0210E0C6E00C10BF0A7EC07F051
:10266000220E0C6E01C10BF0A7EC07F0230E0C6ECE
:1026700002C10BF0A7EC07F0240E0C6E03C10BF0A7
:10268000A7EC07F000C15DF501C15EF502C15FF581
:1026900003C160F55BEF13F004014C0E826FCBECCD
:1026A0000AF00401490E826FCBEC0AF004012C0EF3
:1026B000826FCBEC0AF0250EBEEC07F0E8CF00F1FC
:1026C000260EBEEC07F0E8CF01F1270EBEEC07F0B6
:1026D000E8CF02F1280EBEEC07F0E8CF03F1CBEC17
:1026E00020F0AEEC1EF00401730E826FCBEC0AF00A
:1026F00004012C0E826FCBEC0AF028EC21F0290E9D
:10270000BEEC07F0E8CF00F1CBEC20F0AEEC1EF011
:102710000401730E826FCBEC0AF004012C0E826F61
:10272000CBEC0AF057C500F158C501F159C502F1CB
:102730005AC503F1CBEC20F0AEEC1EF00401730E91
:10274000826FCBEC0AF004012C0E826FCBEC0AF006
:1027500028EC21F05CC500F1CBEC20F0AEEC1EF0D3
:1027600004016D0E826FCBEC0AF004012C0E826F17
:10277000CBEC0AF05DC500F15EC501F15FC502F169
:1027800060C503F182EC1AF004012C0E826FCBECD1
:102790000AF0D5EC0AF067EF1AF083C32AF184C37C
:1027A0002BF185C32CF186C32DF187C32EF188C38D
:1027B0002FF189C330F18AC331F18BC332F18CC35D
:1027C00033F1010176EC21F0EDEC20F0160E0C6EE9
:1027D00000C10BF0A7EC07F0170E0C6E01C10BF057
:1027E000A7EC07F0180E0C6E02C10BF0A7EC07F077
:1027F000190E0C6E03C10BF0A7EC07F000C18AF1B3
:1028000001C18BF102C18CF103C18DF100C18EF1C8
:1028100001C18FF102C190F103C191F1AFEF14F04A
:1028200083C32AF184C32BF185C32CF186C32DF118
:1028300087C32EF188C32FF189C330F18AC331F1E8
:102840008BC332F18CC333F1010176EC21F0EDEC56
:1028500020F000C18AF101C18BF102C18CF103C1EA
:102860008DF100C18EF101C18FF102C190F103C160
:1028700091F1AFEF14F083C32AF184C32BF185C328
:102880002CF186C32DF187C32EF188C32FF189C3A4
:1028900030F18AC331F18CC332F18DC333F10101C0
:1028A00076EC21F0EDEC20F00101000E046F000E3B
:1028B000056F010E066F000E076F3EEC20F01A0E3A
:1028C0000C6E00C10BF0A7EC07F01B0E0C6E01C1E3
:1028D0000BF0A7EC07F01C0E0C6E02C10BF0A7EC7E
:1028E00007F01D0E0C6E03C10BF0A7EC07F000C142
:1028F00092F101C193F102C194F103C195F1AFEFDF
:1029000014F083C32AF184C32BF185C32CF186C351
:102910002DF187C32EF188C32FF189C330F18AC30B
:1029200031F18CC332F18DC333F1010176EC21F02A
:10293000EDEC20F00101000E046F000E056F010E9A
:10294000066F000E076F3EEC20F000C192F101C14E
:1029500093F102C194F103C195F1AFEF14F0160E9B
:10296000BEEC07F0E8CF00F1170EBEEC07F0E8CFA1
:1029700001F1180EBEEC07F0E8CF02F1190EBEEC23
:1029800007F0E8CF03F1CBEC20F0AEEC1EF0040131
:10299000730E826FCBEC0AF004012C0E826FCBEC2D
:1029A0000AF08AC100F18BC101F18CC102F18DC125
:1029B00003F1CBEC20F0AEEC1EF00401730E826F3D
:1029C000CBEC0AF004012C0E826FCBEC0AF01A0E4D
:1029D000BEEC07F0E8CF00F11B0EBEEC07F0E8CF2D
:1029E00001F11C0EBEEC07F0E8CF02F11D0EBEECAB
:1029F00007F0E8CF03F182EC1AF004012C0E826F8D
:102A0000CBEC0AF092C100F193C101F194C102F143
:102A100095C103F182EC1AF0D5EC0AF067EF1AF0D9
:102A20000401690E826FCBEC0AF004012C0E826F58
:102A3000CBEC0AF00101040E006F000E016F000ED6
:102A4000026F000E036FCBEC20F02CC182F4040166
:102A5000300E8227CBEC0AF02DC182F40401300E37
:102A60008227CBEC0AF02EC182F40401300E8227BB
:102A7000CBEC0AF02FC182F40401300E8227CBEC9C
:102A80000AF030C182F40401300E8227CBEC0AF048
:102A900031C182F40401300E8227CBEC0AF032C13E
:102AA00082F40401300E8227CBEC0AF033C182F4A9
:102AB0000401300E8227CBEC0AF004012C0E826F49
:102AC000CBEC0AF00101060E006F000E016F000E44
:102AD000026F000E036FCBEC20F02CC182F40401D6
:102AE000300E8227CBEC0AF02DC182F40401300EA7
:102AF0008227CBEC0AF02EC182F40401300E82272B
:102B0000CBEC0AF02FC182F40401300E8227CBEC0B
:102B10000AF030C182F40401300E8227CBEC0AF0B7
:102B200031C182F40401300E8227CBEC0AF032C1AD
:102B300082F40401300E8227CBEC0AF033C182F418
:102B40000401300E8227CBEC0AF004012C0E826FB8
:102B5000CBEC0AF00101260E006F000E016F000E93
:102B6000026F000E036FCBEC20F02CC182F4040145
:102B7000300E8227CBEC0AF02DC182F40401300E16
:102B80008227CBEC0AF02EC182F40401300E82279A
:102B9000CBEC0AF02FC182F40401300E8227CBEC7B
:102BA0000AF030C182F40401300E8227CBEC0AF027
:102BB00031C182F40401300E8227CBEC0AF032C11D
:102BC00082F40401300E8227CBEC0AF033C182F488
:102BD0000401300E8227CBEC0AF004012C0E826F28
:102BE000CBEC0AF0200EF86EF76AF66A04010900D1
:102BF000F5CF82F4CBEC0AF00900F5CF82F4CBECF0
:102C00000AF00900F5CF82F4CBEC0AF00900F5CF09
:102C100082F4CBEC0AF00900F5CF82F4CBEC0AF099
:102C20000900F5CF82F4CBEC0AF00900F5CF82F46D
:102C3000CBEC0AF00900F5CF82F4CBEC0AF0D5EC2E
:102C40000AF067EF1AF08351630AD8A467EF1AF00D
:102C50008451610AD8A467EF1AF085516C0AD8A490
:102C600067EF1AF08651410A42E08651440A1BE0A0
:102C70008651420AD8B48AEF16F08651350AD8B484
:102C8000F1EF1BF08651360AD8B446EF1CF086519E
:102C9000370AD8B4AFEF1CF08651380AD8B40DEF1C
:102CA0001DF067EF1AF00798079A04017A0E826FF9
:102CB000CBEC0AF00401780E826FCBEC0AF0040131
:102CC000640E826FCBEC0AF081A86EEF16F004015F
:102CD000550E826FCBEC0AF073EF16F004014C0E28
:102CE000826FCBEC0AF0D5EC0AF067EF1AF0078898
:102CF000079A04017A0E826FCBEC0AF00401410EB0
:102D0000826FCBEC0AF00401610E826FCBEC0AF00B
:102D100064EF16F00798078A04017A0E826FCBECF5
:102D20000AF00401420E826FCBEC0AF00401610E3E
:102D3000826FCBEC0AF064EF16F001016667A8EF32
:102D400016F06767A8EF16F06867A8EF16F06967D6
:102D5000C0EF16F04F67B4EF16F05067B4EF16F0FF
:102D60005167B4EF16F05267C0EF16F00101000E84
:102D7000006F000E016F000E026F000E036F120055
:102D80000101620E046F010E056F000E066F000E4A
:102D9000076F66C100F167C101F168C102F169C145
:102DA00003F12DEC20F003BF44EF17F00101000EFA
:102DB000046FA80E056F550E066F020E076F66C1F1
:102DC00000F167C101F168C102F169C103F166C197
:102DD00086F167C187F168C188F169C189F12DEC7D
:102DE00020F003BFFDEF16F00101000E866FA80E64
:102DF000876F550E886F020E896F0E0EBEEC07F0BE
:102E0000E8CF18F10F0EBEEC07F0E8CF19F1100E65
:102E1000BEEC07F0E8CF1AF1110EBEEC07F0E8CFD8
:102E20001BF176EC1FF086C104F187C105F188C162
:102E300006F189C107F12DEC20F007823AEC1FF072
:102E400076EC1FF007923AEC1FF086C100F187C1C3
:102E500001F188C102F189C103F107923AEC1FF038
:102E6000CC0E046FE00E056F870E066F050E076F20
:102E70002DEC20F000C118F101C119F102C11AF1C5
:102E800003C11BF17CEF17F00101800E006F1A0ED9
:102E9000016F060E026F000E036F4FC104F150C1A7
:102EA00005F151C106F152C107F12DEC20F003AF3D
:102EB0005DEF17F028EC21F012000E0EBEEC07F0CB
:102EC000E8CF18F10F0EBEEC07F0E8CF19F1100EA5
:102ED000BEEC07F0E8CF1AF1110EBEEC07F0E8CF18
:102EE0001BF14FC100F150C101F151C102F152C1BA
:102EF00003F107823AEC1FF018C100F119C101F18A
:102F00001AC102F11BC103F112000401730E826F9A
:102F1000CBEC0AF004012C0E826FCBEC0AF0078494
:102F200062C166F163C167F164C168F165C169F1AD
:102F30004BC14FF14CC150F14DC151F14EC152F155
:102F400057C159F158C15AF10794ABEC17F0D5ECC1
:102F50000AF067EF1AF066C100F167C101F168C1BC
:102F600002F169C103F10101CBEC20F0AEEC1EF0DF
:102F70000401630E826FCBEC0AF004012C0E826F09
:102F8000CBEC0AF04FC100F150C101F151C102F187
:102F900052C103F10101CBEC20F0AEEC1EF00401B4
:102FA000660E826FCBEC0AF004012C0E826FCBEC24
:102FB0000AF028EC21F059C100F15AC101F10101D8
:102FC000CBEC20F0AEEC1EF00401740E826FCBEC63
:102FD0000AF0120010820401530E826FCBEC0AF04B
:102FE00004012C0E826FCBEC0AF083C32AF184C358
:102FF0002BF185C32CF186C32DF187C32EF188C335
:103000002FF189C330F18AC331F18BC332F18CC304
:1030100033F1010176EC21F0EDEC20F000C166F116
:1030200001C167F102C168F103C169F18EC32AF1E0
:103030008FC32BF190C32CF191C32DF192C32EF1CC
:1030400093C32FF194C330F195C331F196C332F19C
:1030500097C333F1010176EC21F0EDEC20F000C1D3
:103060004FF101C150F102C151F103C152F169ECBC
:1030700021F099C32FF19AC330F19BC331F19CC366
:1030800032F19DC333F1010176EC21F0EDEC20F03B
:1030900000C159F101C15AF1ABEC17F004012C0E3B
:1030A000826FCBEC0AF05CEF18F08251520A03E118
:1030B0000F825CEF18F00F928251750A03E11084C1
:1030C00063EF18F010948251550A03E110866AEFFD
:1030D00018F01096078410B2C7EF18F010A4B3EFE1
:1030E00018F0B6C166F1B7C167F1B8C168F1B9C1EE
:1030F00069F1BAC16AF1BBC16BF1BCC16CF1BDC170
:103100006DF1BEC16EF1BFC16FF1C0C170F1C1C13F
:1031100071F1C2C172F1C3C173F1C4C174F1C5C10F
:1031200075F1C6C176F1C7C177F1C8C178F1C9C1DF
:1031300079F1CAC17AF1CBC17BF1CCC17CF1CDC1AF
:103140007DF1CEC17EF1CFC17FF1D0C180F1D1C17F
:1031500081F1D2C182F1D3C183F1D4C184F1D5C14F
:1031600085F1BBEF18F062C166F163C167F164C11C
:1031700068F165C169F14BC14FF14CC150F14DC1CE
:1031800051F14EC152F157C159F158C15AF107944A
:103190000FA0E9EF18F001019267D6EF18F09367DE
:1031A000D6EF18F09467D6EF18F09567DAEF18F0BD
:1031B000E9EF18F09DEC16F092C104F193C105F10E
:1031C00094C106F195C107F12DEC20F003BF2DEF5E
:1031D0001AF09DEC16F00101000E046F000E056F51
:1031E000010E066F000E076F5EEC20F010A400EFDA
:1031F00019F00401750E826FCBEC0AF005EF19F09F
:103200000401720E826FCBEC0AF004012C0E826F67
:10321000CBEC0AF0CBEC20F0296714EF19F0040195
:10322000200E826F17EF19F004012D0E826FCBEC88
:103230000AF030C182F40401300E8227CBEC0AF090
:1032400031C182F40401300E8227CBEC0AF0040174
:103250002E0E826FCBEC0AF032C182F40401300EE4
:103260008227CBEC0AF033C182F40401300E8227AE
:10327000CBEC0AF004016D0E826FCBEC0AF0040176
:103280002C0E826FCBEC0AF04FC100F150C101F15E
:1032900051C102F152C103F10101CBEC20F0AEECBF
:1032A0001EF00401480E826FCBEC0AF004017A0E86
:1032B000826FCBEC0AF004012C0E826FCBEC0AF08B
:1032C00066C100F167C101F168C102F169C103F192
:1032D0000101CBEC20F0AEEC1EF00401630E826F16
:1032E000CBEC0AF004012C0E826FCBEC0AF066C125
:1032F00000F167C101F168C102F169C103F1010187
:103300000A0E046F000E056F000E066F000E076FA9
:103310003EEC20F0000E046F120E056F000E066FDB
:10332000000E076F5EEC20F0CBEC20F02AC182F497
:103330000401300E8227CBEC0AF02BC182F4040189
:10334000300E8227CBEC0AF02CC182F40401300E3F
:103350008227CBEC0AF02DC182F40401300E8227C3
:10336000CBEC0AF02EC182F40401300E8227CBECA4
:103370000AF02FC182F40401300E8227CBEC0AF050
:1033800030C182F40401300E8227CBEC0AF0040134
:103390002E0E826FCBEC0AF031C182F40401300EA4
:1033A0008227CBEC0AF032C182F40401300E82276E
:1033B000CBEC0AF033C182F40401300E8227CBEC4F
:1033C0000AF00401730E826FCBEC0AF004012C0E9C
:1033D000826FCBEC0AF028EC21F059C100F15AC100
:1033E00001F191EC1BF00FB2F9EF19F00FA02BEFE8
:1033F0001AF004012C0E826FCBEC0AF0200EF86E4E
:10340000F76AF66A04010900F5CF82F4CBEC0AF002
:103410000900F5CF82F4CBEC0AF00900F5CF82F475
:10342000CBEC0AF00900F5CF82F4CBEC0AF00900EE
:10343000F5CF82F4CBEC0AF00900F5CF82F4CBECA7
:103440000AF00900F5CF82F4CBEC0AF00900F5CFC1
:1034500082F4CBEC0AF0D5EC0AF00F9067EF1AF08B
:103460000401630E826FCBEC0AF004012C0E826F14
:10347000CBEC0AF06DEC1AF004012C0E826FCBEC51
:103480000AF0E0EC1AF004012C0E826FCBEC0AF08B
:103490005CEC1BF004012C0E826FCBEC0AF00101F6
:1034A000F80E006FCD0E016F660E026F030E036FF4
:1034B00082EC1AF004012C0E826FCBEC0AF072EC55
:1034C0001BF0D5EC0AF067EF1AF0D5EC0AF0030117
:1034D000C26B0790109276EF1DF0D8900E0EBEECE6
:1034E00007F0E8CF00F10F0EBEEC07F0E8CF01F1D6
:1034F000100EBEEC07F0E8CF02F1110EBEEC07F0A3
:10350000E8CF03F10101000E046F000E056F010EFC
:10351000066F000E076F5EEC20F0CBEC20F02AC1A6
:1035200082F40401300E8227CBEC0AF02BC182F426
:103530000401300E8227CBEC0AF02CC182F4040186
:10354000300E8227CBEC0AF02DC182F40401300E3C
:103550008227CBEC0AF02EC182F40401300E8227C0
:10356000CBEC0AF02FC182F40401300E8227CBECA1
:103570000AF030C182F40401300E8227CBEC0AF04D
:1035800031C182F40401300E8227CBEC0AF0040131
:103590002E0E826FCBEC0AF032C182F40401300EA1
:1035A0008227CBEC0AF033C182F40401300E82276B
:1035B000CBEC0AF004016D0E826FCBEC0AF0120026
:1035C000120EBEEC07F0E8CF00F1130EBEEC07F0D0
:1035D000E8CF01F1140EBEEC07F0E8CF02F1150EB2
:1035E000BEEC07F0E8CF03F101010A0E046F000EF4
:1035F000056F000E066F000E076F3EEC20F0000E08
:10360000046F120E056F000E066F000E076F5EEC62
:1036100020F0CBEC20F02AC182F40401300E822786
:10362000CBEC0AF02BC182F40401300E8227CBECE4
:103630000AF02CC182F40401300E8227CBEC0AF090
:103640002DC182F40401300E8227CBEC0AF02EC18A
:1036500082F40401300E8227CBEC0AF02FC182F4F1
:103660000401300E8227CBEC0AF030C182F4040151
:10367000300E8227CBEC0AF004012E0E826FCBECC9
:103680000AF031C182F40401300E8227CBEC0AF03B
:1036900032C182F40401300E8227CBEC0AF033C130
:1036A00082F40401300E8227CBEC0AF00401730E81
:1036B000826FCBEC0AF012000A0EBEEC07F0E8CFE6
:1036C00000F10B0EBEEC07F0E8CF01F10C0EBEECE2
:1036D00007F0E8CF02F10D0EBEEC07F0E8CF03F1E2
:1036E00091EF1BF0060EBEEC07F0E8CF00F1070EDD
:1036F000BEEC07F0E8CF01F1080EBEEC07F0E8CF12
:1037000002F1090EBEEC07F0E8CF03F191EF1BF0D8
:10371000010128EC21F0078457C100F158C101F1E3
:1037200007940101E80E046F800E056F000E066F0E
:10373000000E076F3EEC20F0000E046F040E056FC4
:10374000000E066F000E076F5EEC20F0880E046F0F
:10375000130E056F000E066F000E076F2DEC20F0A4
:103760000A0E046F000E056F000E066F000E076F45
:103770005EEC20F0CBEC20F001012967C5EF1BF0D7
:103780000401200E826FC8EF1BF004012D0E826F22
:10379000CBEC0AF030C182F40401300E8227CBEC6E
:1037A0000AF031C182F40401300E8227CBEC0AF01A
:1037B00032C182F40401300E8227CBEC0AF00401FE
:1037C0002E0E826FCBEC0AF033C182F40401300E6E
:1037D0008227CBEC0AF00401430E826FCBEC0AF097
:1037E000120087C32AF188C32BF189C32CF18AC345
:1037F0002DF18BC32EF18CC32FF18DC330F18EC30D
:1038000031F190C332F191C333F10101296B76ECB0
:1038100021F0EDEC20F00101000E046F000E056FA9
:10382000010E066F000E076F3EEC20F00E0E0C6EC0
:1038300000C10BF0A7EC07F00F0E0C6E01C10BF0EE
:10384000A7EC07F0100E0C6E02C10BF0A7EC07F00E
:10385000110E0C6E03C10BF0A7EC07F004017A0EF9
:10386000826FCBEC0AF004012C0E826FCBEC0AF0D5
:103870000401350E826FCBEC0AF004012C0E826F2E
:10388000CBEC0AF06DEC1AF073EF16F087C32AF157
:1038900088C32BF189C32CF18AC32DF18BC32EF180
:1038A0008CC32FF18DC330F18EC331F190C332F14F
:1038B00091C333F10101296B76EC21F0EDEC20F09E
:1038C000880E046F130E056F000E066F000E076F53
:1038D00032EC20F0000E046F040E056F000E066F30
:1038E000000E076F3EEC20F00101E80E046F800E21
:1038F000056F000E066F000E076F5EEC20F00A0EDB
:103900000C6E00C10BF0A7EC07F00B0E0C6E01C1A2
:103910000BF0A7EC07F00C0E0C6E02C10BF0A7EC3D
:1039200007F00D0E0C6E03C10BF0A7EC07F00401BD
:103930007A0E826FCBEC0AF004012C0E826FCBEC76
:103940000AF00401360E826FCBEC0AF004012C0E53
:10395000826FCBEC0AF05CEC1BF073EF16F087C3C0
:103960002AF188C32BF189C32CF18AC32DF18BC3B3
:103970002EF18CC32FF18DC330F18FC331F190C381
:1039800032F191C333F1010176EC21F0EDEC20F03E
:10399000000E046F120E056F000E066F000E076F0B
:1039A0003EEC20F001010A0E046F000E056F000EC0
:1039B000066F000E076F5EEC20F0120E0C6E00C159
:1039C0000BF0A7EC07F0130E0C6E01C10BF0A7EC87
:1039D00007F0140E0C6E02C10BF0A7EC07F0150EE9
:1039E0000C6E03C10BF0A7EC07F004017A0E826F96
:1039F000CBEC0AF004012C0E826FCBEC0AF0040130
:103A0000370E826FCBEC0AF004012C0E826FCBECE8
:103A10000AF0E0EC1AF073EF16F087C32AF188C3BE
:103A20002BF189C32CF18AC32DF18BC32EF18CC3EA
:103A30002FF18DC330F18EC331F190C332F191C3B8
:103A400033F10101296B76EC21F0EDEC20F0880ECA
:103A5000046F130E056F000E066F000E076F32EC39
:103A600020F0000E046F040E056F000E066F000EAE
:103A7000076F3EEC20F00101E80E046F800E056F29
:103A8000000E066F000E076F5EEC20F0060E0C6E47
:103A900000C10BF0A7EC07F0070E0C6E01C10BF094
:103AA000A7EC07F0080E0C6E02C10BF0A7EC07F0B4
:103AB000090E0C6E03C10BF0A7EC07F004017A0E9F
:103AC000826FCBEC0AF004012C0E826FCBEC0AF073
:103AD0000401380E826FCBEC0AF004012C0E826FC9
:103AE000CBEC0AF072EC1BF073EF16F081A834EF08
:103AF0001EF007A8EDEF1DF00101800E006F1A0EF9
:103B0000016F060E026F000E036F4BC104F14CC132
:103B100005F14DC106F14EC107F12DEC20F003BFB8
:103B200034EF1EF0A8EC1EF04BC100F14CC101F1C6
:103B30004DC102F14EC103F107823AEC1FF018C1EA
:103B400004F119C105F11AC106F11BC107F1F80E04
:103B5000006FCD0E016F660E026F030E036F2DEC2A
:103B600020F00E0E0C6E00C10BF0A7EC07F00F0E4C
:103B70000C6E01C10BF0A7EC07F0100E0C6E02C129
:103B80000BF0A7EC07F0110E0C6E03C10BF0A7ECC5
:103B900007F00784010128EC21F057C100F158C15A
:103BA00001F107940A0E0C6E00C10BF0A7EC07F0B0
:103BB0000B0E0C6E01C10BF0A7EC07F00C0E0C6E97
:103BC00002C10BF0A7EC07F00D0E0C6E03C10BF059
:103BD000A7EC07F0079834EF1EF007AA34EF1EF0A9
:103BE0000784010128EC21F057C100F158C101F10F
:103BF0000794060E0C6E00C10BF0A7EC07F0070E41
:103C00000C6E01C10BF0A7EC07F0080E0C6E02C1A0
:103C10000BF0A7EC07F0090E0C6E03C10BF0A7EC3C
:103C200007F0078462C100F163C101F164C102F1D0
:103C300065C103F10794120E0C6E00C10BF0A7ECE6
:103C400007F0130E0C6E01C10BF0A7EC07F0140E79
:103C50000C6E02C10BF0A7EC07F0150E0C6E03C141
:103C60000BF0A7EC07F0079A0401805181197F0B34
:103C70000BE09EA809D014EE00F081517F0BE126E5
:103C8000E750812B0F01AD6E05012F51010A13E0A2
:103C900081AA5BEF1EF005012F51000A0AE00FB860
:103CA0005BEF1EF0050130675BEF1EF00FB85BEFB6
:103CB0001EF0CAEF27F081B870EF1EF058EC22F02A
:103CC00005012F51020A02E070EF1EF05C2F70EF29
:103CD0001EF05BC55CF50501010E306F3C0E316FC7
:103CE0002FEF0AF018C100F119C101F11AC102F158
:103CF0001BC103F1000E046F000E056F010E066F6D
:103D0000000E076F5EEC20F029A19DEF1EF0205100
:103D1000D8B49DEF1EF018C100F119C101F11AC10C
:103D200002F11BC103F1000E046F000E056F0A0EB5
:103D3000066F000E076F5EEC20F0120001010451C7
:103D4000001305510113065102130751031312000A
:103D50000101186B196B1A6B1B6B12002AC182F4DC
:103D60000401300E8227CBEC0AF02BC182F404014F
:103D7000300E8227CBEC0AF02CC182F40401300E05
:103D80008227CBEC0AF02DC182F40401300E822789
:103D9000CBEC0AF02EC182F40401300E8227CBEC6A
:103DA0000AF02FC182F40401300E8227CBEC0AF016
:103DB00030C182F40401300E8227CBEC0AF031C10D
:103DC00082F40401300E8227CBEC0AF032C182F477
:103DD0000401300E8227CBEC0AF033C182F40401D7
:103DE000300E8227CBEC0AF012002FC182F40401BE
:103DF000300E8227CBEC0AF030C182F40401300E81
:103E00008227CBEC0AF031C182F40401300E822704
:103E1000CBEC0AF032C182F40401300E8227CBECE5
:103E20000AF033C182F40401300E8227CBEC0AF091
:103E30001200060E116E060E126E060E136E112E75
:103E40001FEF1FF0122E1FEF1FF0132E1FEF1FF09A
:103E50008B84020E116E020E126E020E136E112E64
:103E60002FEF1FF0122E2FEF1FF0132E2FEF1FF04A
:103E70008B9412000101005305E1015303E1025349
:103E800001E1002BFDEC1FF028EC21F03951006F0F
:103E90003A51016F420E046F4B0E056F000E066F14
:103EA000000E076F3EEC20F000C104F101C105F1E6
:103EB00002C106F103C107F118C100F119C101F1F6
:103EC0001AC102F11BC103F107B26BEF1FF032EC14
:103ED00020F06DEF1FF02DEC20F000C118F101C1B2
:103EE00019F102C11AF103C11BF1120028EC21F0F3
:103EF00059C100F15AC101F1060EBEEC07F0E8CF3E
:103F000004F1070EBEEC07F0E8CF05F1080EBEEC99
:103F100007F0E8CF06F1090EBEEC07F0E8CF07F195
:103F20002DEC20F000C124F101C125F102C126F1E0
:103F300003C127F1290E046F000E056F000E066FF6
:103F4000000E076F3EEC20F0EE0E046F430E056F7F
:103F5000000E066F000E076F32EC20F024C104F152
:103F600025C105F126C106F127C107F13EEC20F07D
:103F700000C11CF101C11DF102C11EF103C11FF1FD
:103F8000120EBEEC07F0E8CF04F1130EBEEC07F002
:103F9000E8CF05F1140EBEEC07F0E8CF06F1150EE0
:103FA000BEEC07F0E8CF07F10D0E006F000E016FB9
:103FB000000E026F000E036F3EEC20F0180E046F2F
:103FC000000E056F000E066F000E076F5EEC20F00E
:103FD0001CC104F11DC105F11EC106F11FC107F18D
:103FE00032EC20F06A0E046F2A0E056F000E066F89
:103FF000000E076F2DEC20F01200BF0EFA6E200E9F
:104000003A6F396BD8900037013702370337D8B091
:104010000EEF20F03A2F03EF20F039073A07035351
:10402000D8B412000331070B80093F6F03390F0B1F
:10403000010F396F80EC5FF0406F390580EC5FF065
:10404000405D405F396B3F33D8B0392739333FA9E2
:1040500023EF20F040513927120001014DEC21F0EF
:10406000D8B01200010103510719346F10EC21F090
:10407000D8900751031934AF800F12000101346B3F
:1040800034EC21F0D8A04AEC21F0D8B012001FEC9B
:1040900021F028EC21F01F0E366F60EC21F00B357B
:1040A000D8B010EC21F0D8A00335D8B01200362FCC
:1040B0004DEF20F034B137EC21F012000101346BE8
:1040C00004510511061107110008D8A034EC21F0A5
:1040D000D8A04AEC21F0D8B01200086B096B0A6B2B
:1040E0000B6B60EC21F01F0E366F60EC21F0075176
:1040F0000B5DD8A488EF20F006510A5DD8A488EFA4
:1041000020F00551095DD8A488EF20F00451085D26
:10411000D8A09BEF20F00451085F0551D8A0053DC1
:10412000095F0651D8A0063D0A5F0751D8A0073D98
:104130000B5FD8900081362F75EF20F034B137EC4B
:1041400021F0346B34EC21F0D89064EC21F007516D
:104150000B5DD8A4B8EF20F006510A5DD8A4B8EFE3
:1041600020F00551095DD8A4B8EF20F00451085D96
:10417000D8A0C7EF20F0003FC7EF20F0013FC7EF06
:1041800020F0023FC7EF20F0032BD8B4120034B167
:1041900037EC21F012000101346B34EC21F0D8B07F
:1041A000120069EC21F0200E366F0037013702371C
:1041B000033711EE33F00A0E376FE7360A0EE75C6D
:1041C000D8B0E76EE552372FDDEF20F0362FD5EF70
:1041D00020F034B12981D890120001010A0E346F09
:1041E000200E366F11EE29F03451376F0A0ED89039
:1041F000E652D8B0E726E732372FF8EF20F0033346
:10420000023301330033362FF2EF20F0E750FF0F77
:10421000D8A00335D8B0120029B137EC21F0120034
:10422000045100270551D8B0053D01270651D8B0EB
:10423000063D02270751D8B0073D03271200005161
:10424000086F0151096F02510A6F03510B6F120081
:104250000101006B016B026B036B12000101046B27
:10426000056B066B076B12000335D8A012000351D3
:10427000800B001F011F021F031F003F47EF21F0AB
:10428000013F47EF21F0023F47EF21F0032B342B92
:10429000032512000735D8A012000751800B041F18
:1042A000051F061F071F043F5DEF21F0053F5DEF6F
:1042B00021F0063F5DEF21F0072B342B072512007C
:1042C0000037013702370337083709370A370B370A
:1042D00012000101296B2A6B2B6B2C6B2D6B2E6B43
:1042E0002F6B306B316B326B336B120001012A5133
:1042F0000F0B2A6F2B510F0B2B6F2C510F0B2C6FA9
:104300002D510F0B2D6F2E510F0B2E6F2F510F0BA9
:104310002F6F30510F0B306F31510F0B316F325106
:104320000F0B326F33510F0B336F120010A806D0F2
:104330008994000EC76E220EC66E05D08984000EC9
:10434000C76E220EC66E050EE82EFED7120010A80C
:1043500002D0898401D08994050EE82EFED7120080
:1043600096EC21F09E96C69E000EC96EFF0E9EB67C
:1043700002D0E82EFCD79E96C69E000EC96EFF0E98
:104380009EB602D0E82EFCD7C9CFABF59E96C69E4E
:10439000000EC96EFF0E9EB602D0E82EFCD7C9CF24
:1043A000ACF59E96C69E000EC96EFF0E9EB602D05C
:1043B000E82EFCD7C9CFADF59E96C69E000EC96EFD
:1043C000FF0E9EB602D0E82EFCD7C9CFAEF59E9662
:1043D000C69E000EC96EFF0E9EB602D0E82EFCD718
:1043E000C9CFAFF59E96C69E000EC96EFF0E9EB653
:1043F00002D0E82EFCD7C9CFB0F59E96C69E000E1F
:10440000C96EFF0E9EB602D0E82EFCD7C9CFB1F51B
:10441000A7EC21F0120096EC21F09E96C69E800E2D
:10442000C96EFF0E9EB602D0E82EFCD79E96C69EA1
:10443000ABC5C9FFFF0E9EB602D0E82EFCD79E96F4
:10444000C69EACC5C9FFFF0E9EB602D0E82EFCD7B3
:104450009E96C69EADC5C9FFFF0E9EB602D0E82E41
:10446000FCD79E96C69EAEC5C9FFFF0E9EB602D073
:10447000E82EFCD79E96C69EAFC5C9FFFF0E9EB61E
:1044800002D0E82EFCD79E96C69EB0C5C9FFFF0E8F
:104490009EB602D0E82EFCD79E96C69EB1C5C9FF37
:1044A000FF0E9EB602D0E82EFCD7A7EC21F012003A
:1044B00096EC21F09E96C69E070EC96EFF0E9EB624
:1044C00002D0E82EFCD79E96C69E000EC96EFF0E47
:1044D0009EB602D0E82EFCD7C9CFABF59E96C69EFD
:1044E000000EC96EFF0E9EB602D0E82EFCD7C9CFD3
:1044F000ACF59E96C69E000EC96EFF0E9EB602D00B
:10450000E82EFCD7C9CFADF59E96C69E000EC96EAB
:10451000FF0E9EB602D0E82EFCD7C9CFAEF5A7ECB1
:1045200021F096EC21F09E96C69E15C0C9FFFF0EA5
:104530009EB602D0E82EFCD79E96C69E000EC96E8F
:10454000FF0E9EB602D0E82EFCD7C9CFB2F5A7EC7D
:1045500021F0120096EC21F09E96C69E870EC96E41
:10456000FF0E9EB602D0E82EFCD79E96C69EABC527
:10457000C9FFFF0E9EB602D0E82EFCD79E96C69EBF
:10458000ACC5C9FFFF0E9EB602D0E82EFCD79E96A2
:10459000C69EADC5C9FFFF0E9EB602D0E82EFCD761
:1045A0009E96C69EAEC5C9FFFF0E9EB602D0E82EEF
:1045B000FCD7A7EC21F096EC21F09E96C69E16C083
:1045C000C9FFFF0E9EB602D0E82EFCD79E96C69E6F
:1045D000B2C5C9FFFF0E9EB602D0E82EFCD7A7ECED
:1045E00021F0120096EC21F09E96C69E870EC96EB1
:1045F000FF0E9EB602D0E82EFCD79E96C69E000EF9
:10460000C96EFF0E9EB602D0E82EFCD79E96C69EBF
:10461000800EC96EFF0E9EB602D0E82EFCD79E9685
:10462000C69E800EC96EFF0E9EB602D0E82EFCD745
:104630009E96C69E800EC96EFF0E9EB602D0E82ED4
:10464000FCD7A7EC21F0120096EC21F09E96C69EB6
:10465000870EC96EFF0E9EB602D0E82EFCD79E963E
:10466000C69E000EC96EFF0E9EB602D0E82EFCD785
:104670009E96C69E000EC96EFF0E9EB602D0E82E14
:10468000FCD79E96C69E800EC96EFF0E9EB602D0C7
:10469000E82EFCD79E96C69E800EC96EFF0E9EB673
:1046A00002D0E82EFCD7A7EC21F0120010A82DD0E4
:1046B00096EC21F09E96C69E16C0C9FFFF0E9EB6D0
:1046C00002D0E82EFCD79E96C69E450EC96EFF0E00
:1046D0009EB602D0E82EFCD7A7EC21F096EC21F094
:1046E0009E96C69E8F0EC96EFF0E9EB602D0E82E15
:1046F000FCD79E96C69E000EC96EFF0E9EB602D0D7
:10470000E82EFCD7A7EC21F0120096EC21F09E9643
:10471000C69E16C0C9FFFF0E9EB602D0E82EFCD77B
:104720009E96C69E010EC96EFF0E9EB602D0E82E62
:10473000FCD7A7EC21F096EC21F09E96C69E910E38
:10474000C96EFF0E9EB602D0E82EFCD79E96C69E7E
:10475000A50EC96EFF0E9EB602D0E82EFCD7A7ECC0
:1047600021F0120096EC21F09E96C69E16C0C9FF5D
:10477000FF0E9EB602D0E82EFCD79E96C69E810EF6
:10478000C96EFF0E9EB602D0E82EFCD7A7EC21F032
:10479000120096EC21F09E96C69E16C0C9FFFF0E31
:1047A0009EB602D0E82EFCD79E96C69E010EC96E1C
:1047B000FF0E9EB602D0E82EFCD7A7EC21F0120027
:1047C00096EC21F09E96C69E910EC96EFF0E9EB687
:1047D00002D0E82EFCD79E96C69EA50EC96EFF0E8F
:1047E0009EB602D0E82EFCD7A7EC21F0120096EC82
:1047F00021F09E96C69E910EC96EFF0E9EB602D007
:10480000E82EFCD79E96C69E000EC96EFF0E9EB681
:1048100002D0E82EFCD7A7EC21F012000501256B91
:10482000266B276B286B899A400EC76E200EC66ECA
:104830009E96C69E030EC96EFF0E9EB602D0E82E4F
:10484000FCD79E96C69E27C5C9FFFF0E9EB602D016
:10485000E82EFCD79E96C69E26C5C9FFFF0E9EB6C3
:1048600002D0E82EFCD79E96C69E25C5C9FFFF0E36
:104870009EB602D0E82EFCD79E96C69EC952FF0E69
:104880009EB602D0E82EFCD7898A0F01C950FF0AD4
:1048900001E1120005012E51130A05E005012E5118
:1048A000170A0CE012000501F00E256FFF0E266FAF
:1048B0000F0E276F000E286F67EF24F00501F00E32
:1048C000256FFF0E266FFF0E276F000E286F899A47
:1048D000400EC76E200EC66E9E96C69E030EC96E13
:1048E000FF0E9EB602D0E82EFCD79E96C69E27C528
:1048F000C9FFFF0E9EB602D0E82EFCD79E96C69E3C
:1049000026C5C9FFFF0E9EB602D0E82EFCD79E96A4
:10491000C69E25C5C9FFFF0E9EB602D0E82EFCD765
:104920009E96C69EC952FF0E9EB602D0E82EFCD7B8
:10493000898A0F01C950FF0A1DE005012E51130A93
:1049400005E005012E51170A0BE012000501000ECB
:10495000256F000E266F100E276F000E286F1200B5
:104960000501000E256F000E266F000E276F010E49
:10497000286F12000501256B266B276B286B05013C
:104980002E51130A05E005012E51170A0CE0120002
:104990000501000E216F000E226F080E236F000E1E
:1049A000246FDCEF24F00501000E216F000E226F52
:1049B000800E236F000E246F21C500F122C501F186
:1049C00023C502F124C503F125C504F126C505F16F
:1049D00027C506F128C507F19EEC1EF000C125F59C
:1049E00001C126F502C127F503C128F5899A400EB9
:1049F000C76E200EC66E9E96C69E030EC96EFF0E33
:104A00009EB602D0E82EFCD79E96C69E27C5C9FF4B
:104A1000FF0E9EB602D0E82EFCD79E96C69E26C5F7
:104A2000C9FFFF0E9EB602D0E82EFCD79E96C69E0A
:104A300025C5C9FFFF0E9EB602D0E82EFCD79E9674
:104A4000C69EC952FF0E9EB602D0E82EFCD7898AB8
:104A5000C950FF0A08E104C125F505C126F506C1C4
:104A600027F507C128F5D8900501243323332233D5
:104A700021332151F00B216F216746EF25F022678A
:104A800046EF25F0236746EF25F02467DCEF24F09E
:104A90000501100E2527E86A2623E86A2723E86A1D
:104AA00028231200E86A05012E51130A06E00501C9
:104AB0002E51170A0BE0020E120005012851000AC0
:104AC00003E12751F00B07E0010E12000501285108
:104AD000000A01E0010E120029C500F12AC501F10A
:104AE0002BC502F12CC503F125C504F126C505F13E
:104AF00027C506F128C507F12DEC20F003BF1200F1
:104B000052EC25F0D8A4E4EF25F0899A400EC76E48
:104B1000200EC66E9E96C69E060EC96EFF0E9EB6EF
:104B200002D0E82EFCD7898A899A9E96C69E020EEC
:104B3000C96EFF0E9EB602D0E82EFCD79E96C69E8A
:104B400027C5C9FFFF0E9EB602D0E82EFCD79E9661
:104B5000C69E26C5C9FFFF0E9EB602D0E82EFCD722
:104B60009E96C69E25C5C9FFFF0E9EB602D0E82EB2
:104B7000FCD79E96C69E000EC96EFF0E9EB602D052
:104B8000E82EFCD7898A899A9E96C69E050EC96E24
:104B9000FF0E9EB602D0E82EFCD79E96C69EC95246
:104BA000FF0E9EB602D0E82EFCD7C9B0CDEF25F09F
:104BB000898A0501100E2527E86A2623E86A27233B
:104BC000E86A28236CEF25F01200899A400EC76E20
:104BD000200EC66E9E96C69E060EC96EFF0E9EB62F
:104BE00002D0E82EFCD7898A899A9E96C69EC70E67
:104BF000C96EFF0E9EB602D0E82EFCD7898A050149
:104C0000256B266B276B286B1200899A400EC76EA6
:104C1000200EC66E9E96C69E050EC96EFF0E9EB6EF
:104C200002D0E82EFCD79E96C69EC952FF0E9EB6B5
:104C300002D0E82EFCD7C9CF33F5898A1200899AB1
:104C4000400EC76E200EC66E9E96C69EB90EC96EE9
:104C5000FF0E9EB602D0E82EFCD7898A1200899AF0
:104C6000400EC76E200EC66E9E96C69EAB0EC96ED7
:104C7000FF0E9EB602D0E82EFCD7898AFF0EE82EE2
:104C8000FED7120052EC25F0D8A41200899A400EEB
:104C9000C76E200EC66E9E96C69E030EC96EFF0E90
:104CA0009EB602D0E82EFCD79E96C69E27C5C9FFA9
:104CB000FF0E9EB602D0E82EFCD79E96C69E26C555
:104CC000C9FFFF0E9EB602D0E82EFCD79E96C69E68
:104CD00025C5C9FFFF0E9EB602D0E82EFCD79E96D2
:104CE000C69EC952FF0E9EB602D0E82EFCD7898A16
:104CF0000F01C950FF0AD8A43DEF27F00501FE0EB1
:104D0000336FB0EC21F0ABC534F5ACC535F5ADC5AE
:104D100036F5AEC537F5AFC538F5B0C539F5B1C50F
:104D20003AF50784B6C166F1B7C167F1B8C168F159
:104D3000B9C169F14BC14FF14CC150F14DC151F1B5
:104D40004EC152F157C159F158C15AF19DEC16F0BC
:104D500000C13BF501C13CF502C13DF503C13EF583
:104D600005015D67BBEF26F05E67BBEF26F05F676E
:104D7000BBEF26F06067BFEF26F0CCEF26F05DC5F5
:104D800004F15EC505F15FC506F160C507F12DECC4
:104D900020F003BF3DEF27F059C13FF55AC140F560
:104DA000B5C541F5B6C542F507940501110E326F40
:104DB000899A400EC76E200EC66E9E96C69E060E3F
:104DC000C96EFF0E9EB602D0E82EFCD7898A899A5A
:104DD0009E96C69E020EC96EFF0E9EB602D0E82EAB
:104DE000FCD79E96C69E27C5C9FFFF0E9EB602D071
:104DF000E82EFCD79E96C69E26C5C9FFFF0E9EB61E
:104E000002D0E82EFCD79E96C69E25C5C9FFFF0E90
:104E10009EB602D0E82EFCD725EE33F0322F02D01A
:104E20001DEF27F09E96C69EDECFC9FFFF0E9EB6F1
:104E300002D0E82EFCD70EEF27F0898A899A9E9639
:104E4000C69E050EC96EFF0E9EB602D0E82EFCD798
:104E50009E96C69EC952FF0E9EB602D0E82EFCD783
:104E6000C9B028EF27F0898A0501100E2527E86AC6
:104E70002623E86A2723E86A2823120021C500F1C7
:104E800022C501F123C502F124C503F1899A400E20
:104E9000C76E200EC66E9E96C69E0B0EC96EFF0E86
:104EA0009EB602D0E82EFCD79E96C69E02C1C9FFD0
:104EB000FF0E9EB602D0E82EFCD79E96C69E01C17C
:104EC000C9FFFF0E9EB602D0E82EFCD79E96C69E66
:104ED00000C1C9FFFF0E9EB602D0E82EFCD79E96F9
:104EE000C69EC952FF0E9EB602D0E82EFCD725EE14
:104EF00033F00501100E326F9E96C69EC952FF0E0A
:104F00009EB602D0E82EFCD7C9CFDEFF322F7CEF51
:104F100027F0898A1200899A400EC76E200EC66E4D
:104F20009E96C69E900EC96EFF0E9EB602D0E82ECB
:104F3000FCD79E96C69E000EC96EFF0E9EB602D08E
:104F4000E82EFCD79E96C69E000EC96EFF0E9EB63A
:104F500002D0E82EFCD79E96C69E000EC96EFF0EAC
:104F60009EB602D0E82EFCD79E96C69EC952FF0E72
:104F70009EB602D0E82EFCD7C9CF2DF59E96C69ED0
:104F8000C952FF0E9EB602D0E82EFCD7C9CF2EF52F
:104F9000898A120019EC1FF0B5C5E8FFD70802E3B3
:104FA00019EC1FF0B5C5E8FFC80802E319EC1FF0C3
:104FB000B5C5E8FFB90802E319EC1FF0B5C5E8FF75
:104FC000AA0802E319EC1FF0B5C5E8FF9B0802E34D
:104FD00019EC1FF058EC22F01FEC26F0F29CF29E28
:104FE0008B94C69AC2909482948C720ED36ED3A482
:104FF000FED789968A909390FF0EE8CF00F0E82EB6
:10500000FED7002EFCD78150F294F29A9E909D908C
:105010009E929D92F298F292F290F286F28E0300A6
:02502000FF008F
:10BF0000E844F926000C160C2B0C3F0C520C640C68
:10BF1000760C860C960CA50CB30CC10CCF0CDC0C6B
:06BF2000E80CF40C000C1B
:00000001FF
